:100000002D28000000000518003414088C0400346A
:10001000140892001508930000341608920017087F
:100020009300003434309200953093000034122055
:1000300020201220202012202020122020200034F6
:100040001208900013089100910B2428900B292886
:100050002C2813089100242800348501860183167A
:100060000514061283121220202001309600193048
:100070009700013094000C30950017208C0101305E
:100080009400051C3E280000000008202020051CCC
:100090003E280D20202001200310940D031C492828
:1000A0000D2020200C08303C03190612031D0616F3
:0600B000122020203E2872
:00000001FF
